:020000040000FA
:10000000B8220020150200001D0200001F0200009F
:100010002102000023020000250200000000000071
:1000200000000000000000000000000027020000A7
:1000300029020000000000002B0200002D02000039
:100040002F0200002F0200005D0400002F020000BC
:100050002F0200002F0200002F0200002F020000DC
:100060002F0200002F0200002F0200002F020000CC
:100070002F0200002F0200002F0200002F020000BC
:100080002F0200002F0200002F0200002F020000AC
:100090002F0200002F0200002F0200002F0200009C
:1000A0002F0200002F0200002F0200002F0200008C
:1000B0002F0200002F0200000000000000000000DE
:1000C0002F0200002F0200002F0200002F0200006C
:1000D0002F0200002F0200002F0200002F0200005C
:1000E0002F0200002F0200002F020000000000007D
:1000F000000000002F020000000000002F0200009E
:1001000000000000000000000000000000000000EF
:1001100000000000000000000000000000000000DF
:1001200000000000000000000000000000000000CF
:1001300000000000000000000000000000000000BF
:1001400000000000000000000000000000000000AF
:10015000000000000000000000000000000000009F
:10016000000000000000000000000000000000008F
:10017000000000000000000000000000000000007F
:10018000000000000000000000000000000000006F
:10019000000000000000000000000000000000005F
:1001A000000000000000000000000000000000004F
:1001B000000000000000000000000000000000003F
:1001C000000000000000000000000000000000002F
:1001D000000000000000000000000000000000001F
:1001E000000000000000000000000000000000000F
:1001F00000000000000000000000000000000000FF
:10020000DFF80CD000F02AF800480047C1080000D1
:10021000B82200200648804706480047FEE7FEE770
:10022000FEE7FEE7FEE7FEE7FEE7FEE7FEE7FEE7A6
:10023000810200000102000040EA01039B0703D095
:1002400009E008C9121F08C0042AFAD203E011F815
:10025000013B00F8013B521EF9D27047064C074D96
:1002600006E0E06840F0010394E807009847103486
:10027000AC42F6D3FFF7C8FF0C1500002C150000A8
:1002800030B54FF0805000228300D0F83011C3F811
:100290000C21C3F81021624B1A60624B1B68624C40
:1002A0002360604B1B1D1B68241D23605D4B0833BE
:1002B0001B68241D23605B4B0C331B68241D2360CB
:1002C000584B10331B68241D2360564B14331B6896
:1002D000241D2360534B18331B68534C2034236078
:1002E000504B1C331B68241D23604E4B20331B686E
:1002F000241D23604B4B24331B68241D2360494B72
:1003000028331B68241D2360464B2C331B68241D97
:100310002360444B30331B68434C40342360414BD3
:1003200034331B68241D23603E4B38331B68241D67
:1003300023603C4B3C331B68241D2360394B403306
:100340001B68241D23600124082902D1D0F8343110
:1003500013B1082904D006E0354B3449196005E093
:10036000D0F8343113B1082904D006E0314BFB2119
:10037000196005E0D0F8343113B1082908D00EE037
:1003800090F858322C48016863F30301016002E0E1
:10039000D0F834311BB929494FF40070086028485F
:1003A0000168C90702D06FF00101016025480168AA
:1003B00041F470010160BFF34F8FBFF36F8F4FF0B7
:1003C0001021D1F80002002803DBD1F80402002834
:1003D00022DA1D4B1C601D480468002CFCD012243E
:1003E000C1F800420568002DFCD0C1F80442016844
:1003F0000029FCD01A6001680029FCD0BFF34F8FA0
:1004000010487C380168124A01F4E0611143016030
:10041000BFF34F8F00BFFDE70F490E48086030BDA6
:10042000380500400404001020C500404881030046
:100430008C56004018F50040E40E00404096024003
:100440000004004088ED00E004E5014000E40140C4
:100450000400FA050090D003400000200148006825
:100460000047000014000020014A024900F013B8C0
:10047000310800003C00002002E008C8121F08C13B
:10048000002AFAD170477047002001E001C1121F15
:10049000002AFBD170472DE9F04116460F4604466D
:1004A000002503E03946B047641C6D1C2078002805
:1004B000F8D12846BDE8F08172B609480068C00747
:1004C00000D000BEBFF34F8F0548E4380168054AED
:1004D00001F4E06111430160BFF34F8F00BFFDE7FE
:1004E000F0ED00E00400FA050EB500210091CDE921
:1004F00001106A4644F20100FFF7DEFF0EBD10B5A1
:100500008268C368934203D000F07FF9002010BDD9
:10051000052010BD29B112B1531E134203D009208A
:1005200070470E2070470160838000218160C160A8
:100530000846704710B58268C3689A1A83889A4241
:1005400003D800F06CF9002010BD042010BD00009D
:1005500070B50A4E01460A48B578FFF7D0FF044649
:100560004DB10020B070711C0122C81D00F02AFAA4
:1005700008B1FFF7B9FF204670BD00001C00002045
:1005800094020020F0B5244E89B01F460D000446A9
:1005900072603FD0A888296882B22048FFF7BAFF6E
:1005A000002835D1A889A96882B21C481030FFF70D
:1005B000B1FF00282CD1202219496846FFF73CFEE4
:1005C00060690690207C00B101208DF814008DF840
:1005D0001C70607C00B10E208DF81500E068029060
:1005E000A068039020680190606800900A480D4A56
:1005F0006946083000F0B2F9002809D1B0702068CF
:10060000401C05D004490122491CC81D00F0DAF93C
:1006100009B0F0BD0720FBE71C0000209402002079
:10062000EC140000A911000010B501461048FFF7B6
:1006300081FF040019D10F480F4A0178515C19B1AC
:10064000001D00F031FD02E00C3000F015FC60B937
:10065000084907480839FFF752FF30B90549012218
:100660000839044800F0BEF90446204610BD0000D9
:10067000A4020020240000200000002000F002B8A6
:1006800000F008B872B602480168491C0160704762
:100690003800002003490868401E086000D162B697
:1006A000704700003800002070B5054608680C4609
:1006B000411C04D000F042FA206800F000FA6068A3
:1006C000411C02D0002100F0E8F92968A069C1F8B6
:1006D0002405607D227D29681043C1F86C05D4E9AA
:1006E00000122868C0F81425C0F80C15207D0128D8
:1006F00014D1A068411C02D0002100F0CEF9E068BE
:10070000411C04D000F01AFAE06800F0D8F9D4E9EE
:1007100002122868C0F80825C0F8101570BD70B521
:10072000054608680C46411C04D000F011FA206808
:1007300000F0CFF96068411C02D0002100F0B6F94A
:100740002968A069C1F82405607D217D2A680843D5
:10075000C2F86C05D4E900122868C0F80C15C0F87E
:100760001425207D012814D1A068411C02D000214D
:1007700000F09CF9E068411C04D000F0E9F9E06861
:1007800000F0A7F9D4E902122868C0F80825C0F8DB
:10079000101570BD2DE9FC410646C0074FF000055D
:1007A0000ED0104F00240122385D00950023114621
:1007B000019500F027F9641C042CF4D300F01CF818
:1007C000B0070DD5074E0024361D0022305D0323EF
:1007D00000951146019500F015F9641C042CF4D322
:1007E000BDE8FC81DC1400000249085C012100F036
:1007F000B9B90000DC14000010B500242046FFF752
:10080000F3FF641C042CF9D310BD826883881A405E
:1008100003689A5C0A708168491C81607047C268ED
:1008200083881A4003689954C168491CC1607047A5
:1008300010B50446C0B2FFF7F7FE204610BD000019
:1008400070B50D46044600684FF4887100F0B3F9A6
:100850004FF49071206800F0AEF94FF49271206867
:1008600000F0A9F94FF4A271206800F0A4F9206803
:100870001249C0F8041320686907000B40B2090E42
:10088000002806DA00F00F0000F1E02080F8141DC7
:1008900003E000F1E02080F8001420680121000B43
:1008A00040B200F01F0291404009800000F1E020BA
:1008B000C0F88012C0F8001170BD000010030200E3
:1008C0008AB00120FFF766FF182216496846FFF735
:1008D000B3FC1548069015494FF48070CDE9070127
:1008E00009900723124A06A96846FFF74BFE08B194
:1008F000FFF7FAFD0FA0FFF7B7FD06A8FFF728FEE8
:100900000028FAD19DF81800FFF78EFE0028F9D1D3
:100910009DF81800712801D05128EED10CA0FFF7E6
:10092000A3FDFEE7C41400004400002044010020A1
:10093000971100000D0A55415254206578616D7081
:100940006C6520737461727465642E0D0A0000007A
:10095000200D0A45786974210D0A0000F0B505469E
:100960000478154889B0164640F82420124A0869D0
:100970000832A2F10C0742F82400487F38552022A3
:100980006846FFF759FC04942878385C48B10EB1EA
:100990000A4A00E000226946281D00F085FA09B0E5
:1009A000F0BD0EB1064A00E00022694605F10C00D8
:1009B00000F030F9F3E7000004000020A11300006C
:1009C0004912000030B40378054CE35C1BB130BC25
:1009D000001D00F09FBA30BC0C3000F085B900005B
:1009E0000000002030B40378054CE35C1BB130BC40
:1009F000001D00F011BB30BC0C3000F0EBB9000062
:100A0000000000202DE9FF411C46DDE90A7815466B
:100A10000E46684600F068F846EA450141EA84015E
:100A200041EA072242EA0841009A00EB8200C0F83E
:100A30000017BDE8FF812DE9FF411C46DDE90A787A
:100A400015460E46684600F05DF846EA450141EA63
:100A5000840141EA072242EA0841009A00EB820041
:100A6000C0F80017BDE8FF812DE9FF411C46DDE914
:100A70000A7815460E46684600F052F846EA4501E7
:100A800041EA840141EA072242EA0841009A00EB68
:100A90008200C0F80017BDE8FF811CB500220B469C
:100AA000009211460192FFF7C6FF1CBD1CB5002243
:100AB0000B46009211460192FFF7D6FF1CBD1CB5F4
:100AC000002100910B46012201911146FFF7B3FF6F
:100AD0001CBD1CB5002100910B460122019111465D
:100AE000FFF7C2FF1CBD00000168202902D24FF0B1
:100AF000A040704701F01F010160014870470000ED
:100B0000000300500168202902D24FF0A040704736
:100B100001F01F0101600148704700000003005010
:100B20000168202902D24FF0A040704701F01F0158
:100B300001600148704700000003005001B568469D
:100B4000FFF7E0FF009A01219140C0F8081508BDA9
:100B500001B56846FFF7E4FF009A01219140C0F813
:100B6000081508BD38B501240090684631B1FFF77B
:100B7000BBFF00998C40C0F8084538BDFFF7B4FFB3
:100B800000998C40C0F80C4538BD4058002800D072
:100B90000120704708B5002242504058009008BD1F
:100BA000D0F80403084000D00120704740580028C6
:100BB00000D00120704708B50022425040580090F4
:100BC00008BD0121B1EB507F01D101207047002009
:100BD000704770B50D4600F075FA04000FD0002084
:100BE000FFF74CFD207920B10020FFF749FD1120CF
:100BF00070BD0120256020710020FFF741FD00201D
:100C000070BD00000149024800F036BB44020020DC
:100C1000002000402DE9F0410546007916460F46B8
:100C200000EB40012D4A01EBC00102EB810494F876
:100C30002A1011B10820BDE8F081294951F820108F
:100C40002868FFF7C6FF08B11120F4E739462846A7
:100C5000FFF72AFD66603869206030004FF001061A
:100C60002FD03F7F4FF48E712868FFF793FF4FF42A
:100C7000A2712868FFF78EFF28681A49C0F804138C
:100C800028684FEA4711000B40B2002806DA00F04E
:100C90000F0000F1E02080F8141D03E000F1E020D7
:100CA00080F800142868000B40B200F01F0206FA1A
:100CB00002F14009800000F1E020C0F88012C0F885
:100CC000001128680421C0F800150020A061E0612F
:100CD00084F8290044F8140FA675ACE744020020FC
:100CE000E4140000800002002DE9F05F0546007961
:100CF0004FF4017600EB400303EBC000344B03EBF1
:100D000080040020636813B12B68C3F80863A369EB
:100D10004FF000096BB1E06938B1606810B1286824
:100D2000C0F804631120BDE8F09FE2610120216159
:100D300005E0C4F82490A261E160C4F81C9094F826
:100D40002910014302D1284600F0F8F96068002814
:100D5000286803D0C0F804630020E4E74FF4A276CB
:100D60003146FFF717FFB2464FF4927B5946286889
:100D7000FFF70BFF06464FF484712868FFF705FF65
:100D8000804651462868FFF700FF074648EA0700FB
:100D90003043EBD056EA070007D12146286800F01F
:100DA0009DF9A169606A8142E0D8C4F818900EB13B
:100DB0000320B8E70FB10F20B5E794F82910012000
:100DC0000029296801D00860C6E74860C4E7000030
:100DD000440200202DE9F047054600790B4600EB60
:100DE000400101EBC000234901EB8004284600F0DC
:100DF00043F810B11120BDE8F0874FF00008C4F8A7
:100E00002080A360626184F828804FF48E76474684
:100E100031462868FFF7BEFE28684FF00109C0F888
:100E200008902146286800F099F9606800BBD5F861
:100E300000A00EE094F8280008B10F2716E0314614
:100E40005046FFF7A2FE0028F4D02146504600F09D
:100E500085F9216A60698142F1D331462868FFF73C
:100E600094FE0028F9D02868C0F80C90C4F81480CB
:100E70003846C0E744020020007900EB400101EB56
:100E8000C000044901EB80004069002800D0012027
:100E900070470000440200200149024800F098BA5F
:100EA00070020020002000402DE9F0410546164662
:100EB00000790F46154A00EBC00102EB810494F85B
:100EC000201011B10820BDE8F081114951F820101F
:100ED0002868FFF77EFE08B11120F4E7394628465E
:100EE000FFF71DFC6660386920601EB1397F284617
:100EF000FFF7A6FC28680821C0F800150020A061B3
:100F0000E0610121606184F82010DCE770020020BC
:100F1000E81400002DE9F05F044600790E4600EB6E
:100F2000C001DFF8F0A017460AEB81053046FFF755
:100F300048FEB0B168684FF000084FF4047910B172
:100F40002168C1F80893A8694FF0000B80B1E869E7
:100F500048B1686810B12068C0F804931120BDE85A
:100F6000F09F1020FBE7EF614FF001082E6102E0D7
:100F7000EE60C5E9067B00254FF488712068FFF715
:100F80001AFE4FF4A2712068FFF715FE2068C0F822
:100F90003465C0F838752068B8F1000F12D0D0F869
:100FA000001241F02001C0F800122079D04600EB79
:100FB000C0010AEB8100406838B12068C0F8049392
:100FC0002846CCE701210160EFE74FF4887A4FF41F
:100FD000A27951462068FFF7E9FD07464946206897
:100FE000FFF7E4FD06464FF492712068FFF7DEFD3F
:100FF000014647EA06000843EBD0227902EBC20320
:1010000008EB8302C2F818B001B10325002ED7D037
:101010000F25D5E7700200202DE9F04704460E4663
:101020000079204900EBC00001EB800517463046EF
:10103000FFF7C7FD30B1204600F036F820B111208F
:10104000BDE8F0871020FBE76F61AE604FF490764B
:10105000002731462068FFF7AEFD4FF4AC784146DB
:101060002068FFF7A8FD2068AA686969C0F84425D0
:10107000C0F84815206801218160686878B9B146D8
:1010800049462068FFF792FD064641462068FFF773
:101090008DFD0643F4D000B10F270020686138466B
:1010A000CEE70000700200200079054900EBC00087
:1010B00001EB80004069002800D00120704700004B
:1010C000700200200349884201D103487047002084
:1010D00070470000002000401400002070B5054655
:1010E00088690C4600284FF4847128460AD0FFF71F
:1010F00051FDD5F81805626AE1688854606A401CA1
:10110000606270BDFFF746FDD5F8180570BD1FB5CC
:1011100001238DF80030CDE90121D0E900126846A5
:1011200090471FBD1FB501238DF800308DF80810C2
:101130000192D0E90012684690471FBD10B50446E1
:1011400000684FF49271FFF725FD4FF48471206819
:10115000FFF720FD20680121016010BD70B50C462D
:1011600005464FF48E71FFF715FD216AA068415CBA
:10117000206A401C2062C5F81C1570BD1FB50022F6
:101180008DF800200291816801914261D0E900123E
:10119000684690471FBD0178022901D0012902D17C
:1011A0004068FFF7A1B970477CB50178244D81B341
:1011B00001290BD002292BD18DF80010C068691CC1
:1011C00001900122C81DFFF7FDFB2EE04068017869
:1011D0001C48FFF7AFF91B4C012618B18DF80060D1
:1011E000019006E0A068E168814205D000208DF8FA
:1011F0000000696868468847A068E168081AA18805
:10120000884207D80E490122491CC81DFFF7DAFBA6
:101210007CBD01E0AE70FBE70A4809491030FFF7DA
:101220006EF930B103208DF8000069686846884780
:10123000EEE70349012201F10800FFF7D3FBE7E7DE
:101240001C000020940200201FB50A4601788DF88A
:10125000001041680191017A8DF80810C068039070
:10126000044850F82210083850F822206846904769
:101270001FBD00000C0000202DE9FF470C4605466D
:101280004FF40071FFF78CFC01274FF40178002622
:1012900018B34FF4927949462846FFF776FCE0B13F
:1012A00049462846FFF776FCC5F8088394F82900DC
:1012B00000B96F6002208DF80000D5F88004C5F8F1
:1012C00080040390A0690290E0680190A661E66145
:1012D000D4E900126846904728E004212846FFF729
:1012E0005FFC18B34FF484712846FFF74EFCE8B159
:1012F00021462846FFF7F2FE616AA069884215D1AF
:10130000E06938B1E268616AA0612069E6616662FD
:10131000E06008E094F8290000B96F60C5F8088320
:10132000A661E268616A2046FFF7F1FE4FF48E780D
:1013300041462846FFF729FC78B1206A6169884256
:1013400002D294F8280020B341462846FFF722FC39
:10135000616911B12046FFF711FF4FF4A2784146B1
:101360002846FFF712FC002818D041462846FFF710
:1013700011FC94F8290000B12F60A06900280DD05D
:10138000A661E268616A04B02046BDE8F047FFF755
:10139000BEBE21462846FFF7E1FEDEE7BDE8FF8737
:1013A0001FB50A4601788DF8001041680191017A55
:1013B0008DF80810C0680390044850F822100838CF
:1013C00050F82220684690471FBD00000C00002006
:1013D0002DE9FF410C464FF4927705463946FFF759
:1013E000E5FB0026C0B139462846FFF7E4FB0220A2
:1013F0008DF80000D5F88004C5F880040390D5F876
:101400003C058DF80800E0680190A661E661D4E92A
:1014100000126846904723E04FF488773946284603
:10142000FFF7C4FBE0B139462846FFF7C4FBD5F807
:101430003C15A069884213D1E06960B1E268D5F833
:10144000000220F02000C5F80002E069A0612069D8
:10145000E661E06001E0A661E2682046FFF762FE17
:101460004FF4A27739462846FFF7A0FB60B1394612
:101470002846FFF7A0FBA06930B1A661D5F83C155E
:101480002046E268FFF74EFE4FF490773946284633
:10149000FFF78CFB002813D039462846FFF78BFB5B
:1014A000606900280CD0D5F84C058DF800608DF8E7
:1014B0000800A06801906661D4E900126846904770
:1014C000BDE8FF81080000000600000005000000E4
:1014D000070000000000000000E0D7010D0E0F1013
:1014E0000B0C1819050C0000990E0000FFFFFFFF00
:1014F000FFFFFFFFFFFFFFFFFFFFFFFF00000000F8
:10150000000000000000D601070100002C150000BB
:101510000000002044000000780400007015000066
:101520004400002074220000880400000000000035
:1015300000000000000000000000000000000000AB
:10154000000000000000000000000000000000009B
:1015500000000000002000400000000000200040CB
:101560000000000000000000000000000090D00318
:0400000500000201F4
:00000001FF
